:10380000023FC700E575645A600280FEE4900051F3
:10381000F0752B0679FEE52D245FB40B0040030202
:103820003B6E90383075F003A4C58325F0C58373D3
:10383000023851023B610239E002399002387502C8
:10384000390F023AA5023A600239CC02387B0239BC
:103850005EA9A1E4FBEB903E6593FF74322BF8E682
:103860006F600579F1023B6E0BBB10E9900051745B
:1038700011F0023B6E300003023B87E52E24FBF57E
:103880000AE531FEE530FDEEF50BEDF50CE52D64B6
:10389000A5704FFBEBC3950A4003023B6EEB7E0025
:1038A000250CFFEE350BFEEEC0E0EFC0E0EB540759
:1038B000FD2423F8E6FF74362BF8E66FFE74222D04
:1038C000F8E6FD74352BF8E66DFDEEFCD0E0FFD098
:1038D000E0FE123EACC9EFC9E96003023B6E0B0B80
:1038E00080B2E4FBEBC3950A4003023B6EE50C2B70
:0F38F000FFEB54072422F8E6FE74352BF8E66E42
:1038FF00FD123F7AC9EFC9E96003023B6E0B80D519
:10390F00E52E24FBF50A54076003023B6EE531FEFA
:10391F00E530FDED8E73F574E4FBEBC3950A502A89
:10392F00EB54072422F8E6FF74352BF8E66FFF857A
:10393F007482857383E4936F600579F5023B6E059E
:10394F0074E574700205730B80D0E4F9023B6EE5E9
:10395F0034252BF52B7585C07B06EBC3952B501C9F
:10396F00E5302B24FA25E0F58475868E744C2BF503
:10397F0082E43400F583E58EF00B80DEE4F9023B40
:10398F006EE530C394085003023B6E753004E4F5C6
:10399F000BF50C74FFFDFCAF0CAE0B123EACC9EF78
:1039AF00C97404250CF50CE4350BF50B5403450CC9
:1039BF0070021530E53070DBC200023B6EE4FBCFC6
:1039CF00EBCF7DFF123F7AC9EFC90BBB80F1023BF2
:1039DF006EE52EC3941E5003023B6EE52E75F00765
:1039EF0084FB25E025E02430F8E66570F52274307D
:0239FF002BF8A3
:103A0100E66570F524EB75F006A42430F8E66570E0
:103A1100F525EB75F003A42430F8E66570F526EB87
:103A210075F005A42430F8E66570F528E52E75F0EB
:103A31000584FB2430F8E66570F523EB75F003A4EB
:103A41002430F8E66570F527E5A12522F529E4FB88
:103A5100F974222BF8E629F90BBB08F5023B6EE558
:103A610030540764076003023B6E533B7F433B4086
:103A7100FBEB24F0FFE4343FFEEEC0E0EFC0E07466
:103A8100332BF8E6FE74322BF8E6FDEEFCD0E0FFB6
:103A9100D0E0FE123EACC9EFC90B0BEBC3940A4058
:103AA100D0023B6EE4F9E53054076407703F7907B3
:103AB10075733F7574F0FB857482857383E493FF9E
:103AC100744C252BF582E43400F583EFF00574E5A1
:103AD1007470020573052B0BBB0ADC052B052B90BB
:103AE1000056E054DFFFF0E5B154204FF0E53030EF
:063AF100E31FC94408C9EF
:103AF700E4FBEB903EA893FF744C252BF582E4344E
:103B070000F583EFF0052B0BBB04E7E53030E43C11
:103B1700C94410C975733F7574FCE4F570FB85746F
:103B270082857383E493FF744C252BF582E434007C
:103B3700F583EFF0052B2570F5700574E5747002B9
:103B470005730BBB04D87404252BF52B75A155758C
:103B5700A1AA75B10CE4F5A1800DE530B40104D23A
:103B6700018002D200E4F990004CE52DF0E52B240A
:103B7700FC90004EF0E4A3F0A3E9F0E4F575F52A14
:103B87002220D903023C99E5D9543F7003023C93A4
:103B970024E07003023C7324FE603824F2603F2463
:103BA7002E6003023C9620DE03023C9685DB0975F6
:103BB7000D01750E00750F0C8509107B007A0079D1
:103BC7002D123F1B75755A123804852BD553D4FC1B
:103BD700023C96E5D454FC4402F5D4023C96E5DB5E
:103BE70064087069900006E0F52CC203900000E0BD
:103BF70054606004D2038057900001E0F56FE56FD1
:103C070024FB603024FD602E1460362403703A9044
:0A3C17000003E024FE600E047016A6
:103C210075713E757276750912802A75713E7572CD
:103C310088750920801FD203801B800B900000E54E
:103C410021F0750901800E900002E0F5218006D275
:103C5100038002D203300308756FFF75DCCF803516
:103C6100E52CD39509400385092C123EE475DCC08F
:103C71008023E56F24FB600B147012123EE463DCB9
:103C8100408012E5E354804521F5E38005E4F5DD4C
:103C9100800075DC02C2D92230D80B75DC0275D4E4
:103CA10012E4F5E3800630DA03C2DA2275D8FF2286
:103CB10075A15575A1AAE5B954F84404F5B9C20135
:103CC100D200E5A1139202C2AFC28CC28D3002169E
:103CD100759850E4F5C875878075892075C9A075F8
:103CE1008DF3D28E800675C03075C2F3903FF4E437
:103CF10093FF30E107A2B6E433FE80093095047EDC
:103D01000080027E01EE7013E5B130E50E900000F7
:103D1100E493B4FF23A3E493B4FF1DE4F5E275EB50
:103D21000CF5EDF5ECF5E575E40C75E22975D1813D
:103D310075D8FF75E1078013EF30E00D43890175F8
:103D41008AC0758C64D28C8002D201E4F508123EDF
:103D51001874222508F8C6EFC60508E508C39408BB
:103D610040EC30010B75A15575A1AA75B11080FE0B
:103D710020C003309806752A96123D94E5D8540761
:103D81006006752A96123B88308DD7C28DC28CD2BF
:103D91000180CF123FB4EF6457707B123FB4EF64E0
:103DA100AB7073123FB48F2DAE2D123FB48F2EE541
:103DB1002E2EFE123FB48F2FE4FDED652E600E1204
:103DC1003FB474302DF8EFF62EFE0D80ED123FB4A6
:103DD100EF6E7042C28CC28D75755A123804E4FEC2
:103DE1007F55123F9D7FAA123F9DFDEDC3952B503C
:103DF1001F744C2DF582E43400F583E0FF123F9DE2
:103E0100744C2DF582E43400F583E02EFE0D80DB49
:103E1100CFEECF123F9D22AC11AD12AE13AF14788D
:103E210010EC4D4E4F70047CA57DA5C3EC13FCED49
:103E310013FDEE13FEEF13FF5010EC64CCFCED64A8
:103E41004CFDEE644EFEEF64CEFFD8DF8C118D1277
:103E51008E138F14EE547FFE228E118F1274A5F5EE
:103E610013F514224D435520495350202620574322
:103E7100482E434E0012011001FF8055084843E0CF
:103E810055000100000001090220000101008032FB
:103E91000904000002FF805500070582024000006E
:0B3EA1000705020240000000020301C0
:103EAC00E52A6496600280FEC3EE94384011EF94CC
:103EBC00F0EE943F401FD3EF94F8EE943F50168EE3
:103ECC00858F848C8F8D8EE58630E60975869AE514
:103EDC00866440FF227F4022E52CC3940840047F77
:103EEC00088002AF2CCEEFCE750DFF85710E85725A
:103EFC000F8E107B017A007900123F1BC3E52C9EBC
:103F0C00F52CEE2572F572E43571F5718EDD228B90
:103F1C000A8A0B890CAF101510EF6026AB0D050F3C
:103F2C00E50FAA0E7002050E14F9123F4FFFAB0AF3
:103F3C00050CE50CAA0B7002050B14F9EF123F6887
:103F4C0080D322BB010689828A83E0225002E722B9
:103F5C00BBFE02E32289828A83E49322BB01068999
:103F6C00828A83F0225002F722BBFE01F322E52A5B
:103F7C006496600280FE7585C0EF25E0F5848D8E19
:103F8C00E58630E60975869AE5866440FF227F4017
:103F9C002230020AC2998F993099FDC29922C2C16E
:103FAC008FC130C1FDC2C1223002083098FDC298C9
:103FBC00AF992230C0FDC2C0AFC122787FE4F6D8E1
:073FCC00FD758175023CB197
:043FF40003000000C6
:00000001FF
